:1074000080E189BD82E189BD09B400FEFDCF089508
:10741000AA2069F08091E9008F931092E9009BD433
:1074200083FF01C01AD58F9187708093E90008957A
:107430008EEF0090E10008220092E1000895F20131
:10744000F999FECFF2BDE1BD0895F9DFF89A80B554
:1074500008C0F5DF1FBA80BD0FB6F894FA9AF99A02
:107460000FBE31962F010895E0E0F0E085919491F0
:10747000019608958BEA34D0109289008AEF8093A8
:10748000880082E080936F0083E080938100EDE9C3
:10749000F7E7859130D0E93AE1F781E08093D700B2
:1074A0008AE482BF1092D8001092E2001092DA00B3
:1074B0001092E10080E808D019BCAA241092E000E4
:1074C00060D489E051D481E98093D8000895A3E67F
:1074D000B1E090E810D08D939A95E1F7089586E099
:1074E00008D015C083E005D08F2F05D08E2F03D094
:1074F00080E05E9A72988EBD8DB587FFFDCF8EB508
:10750000089505D085E0F5DFF6DF80FDFDCF729AA6
:107510005E9808958FE08221E9F7F9DFE3E6F6E06F
:1075200090EB5C98892FE7DF80E1E5DF5C9A819141
:10753000E2DF83E68E278F77D1F79395983B89F723
:107540000895E3E6F1E097FC36C094FC4DC092FE4E
:10755000089596849920D1F3F894C089D78520E0C6
:1075600030E080E090E4AFEFBFEF119689199040D2
:10757000E0F72D01BD4F8D0127FD13C0E0E0F8E0DD
:1075800011928EE7819392E4E11791939AE508F0C6
:1075900092E4E334C9F781931082BFDFFE012196A4
:1075A000A1DF95DFF901FBD420583F4F040D151DD5
:1075B0009A9411F710C28301282D60906C0170908D
:1075C0006B0143D019F48823C1F70895380188244A
:1075D0003CD0C9F580916A01821709F4830160905B
:1075E0006E0170906D01F4CF80E1982E60906E0175
:1075F00070906D012AD059F48823B1F708959FEF58
:1076000095FC03C096FE089591E097FB890E6624D1
:1076100077248301222719D0B1F48823A1F3809124
:107620006A0136F0881650F4821730F0213003C01A
:10763000881520F4281710F48301282F60906E011C
:1076400070906D01E8CF3801822EF3014BDF3FDFF0
:10765000C3E6D1E0E6E9F7E709908591081621F441
:10766000ED39D1F70880801052CFC9E032DFCA95DA
:10767000E9F7D0E195FC1EC094FC37C096FE51C0DE
:10768000C3E6D2E0E3E6F6E098E088E78E0F0084F8
:107690000192E817E1F7884F09900192E817E1F7A6
:1076A000C858DF4F9A9589F735DFC85FD340C33E8E
:1076B00049F749C0C3E6D6E0EBE5FAE098E08E2F43
:1076C000885702900086E817E1F738960A900292F0
:1076D000E817E1F73897C857D0409A9581F71ADF35
:1076E000C850DC4FC33E41F72EC0A3EEB6E0E3E640
:1076F000F6E09AE0C6E00D9080818025807F8025AD
:1077000082958193A336B90709F4B2E0E336F9070D
:1077100009F4F2E0E336FC0771F7FCDEDA9529F7AD
:1077200012C0A3EEB9E0E3E6FAE092E00E90829197
:1077300080258F70802582958083E336F907B1F725
:10774000E9DEDA9571F78827089580E880BF8DEA31
:107750008093640089E98093650085E083BF889504
:10776000E8EBF0E081818C7F81838CE0808374E0A2
:10777000720D84EA02C0838384E88483848187FD58
:1077800008957211FBCF089502D084E9848388E0C4
:107790008A95F1F7089541524455424F59D5F08DDD
:0A77A00014A1C881CFD9F1AF000099
:1077AA001201100102000008412336000100000006
:1077BA00000109023E0002010080320904000001B2
:1077CA000202010005240010010424020405240613
:1077DA000001070582030800FF09040100020A00EC
:1077EA0000000705040210000107058302100001CA
:1078000011241FBE04B714BE88E1E0E6F0E08083D7
:1078100011928EEF9AE09EBF8DBF22243324210166
:1078200031014101510187C00F928F939F931F92A5
:107830000FB60F9211244F936F938091DA0080FF5F
:1078400034C020C00F920FB68F939F93EF93FF9396
:1078500088278093850080938400E0E5F1E09081A3
:107860008917980B908309F45D9A91818917980B79
:10787000918309F4289A239411F48315381EFF91FB
:10788000EF9154C08091D80080FF0FC08091DA0042
:107890008E7F8093DA008091D90080FF04C0B0DD34
:1078A00081E0A82E02C019BCAA248091E10080FFCB
:1078B0000BC054D280FF08C054D28091D80080629F
:1078C00003DE19BC85E0A82E8091E10084FF1AC078
:1078D00045D284FF17C094DD8091D8008F7DF4DD00
:1078E0008FEEA7DD3BD28F7E81603ED28091530127
:1078F000882331F48091E30087FD02C081E001C05C
:1079000084E0A82E8091E10083FF0CC027D283FF82
:1079100009C087EF8EDD82E0A82E1092530188DD2A
:1079200020D22FD26F914F910F901F909F918F91E6
:107930000FBE0F90189580E880831082B1E0B5BF2C
:1079400082E085BF81EF85B987EE84B984E08DB987
:1079500084E48EB910BA83EF81BB80E68BB980EFE7
:107960008AB980E58CBDBDBDA0E0EAEAF7E70590E5
:107970000D92A035E1F78C911D92BB30E1F7893B68
:1079800011F4AEDDE2CE5F9A00FD7C9B02C06CDD9F
:1079900011F570DD789459DEB4D03ADD8FB1809561
:1079A000807F66991C9B8460982E29DE89EB882550
:1079B0008093FF0A8110C5DD882049F492FC09C03C
:1079C0008FE0822121F48091720187FF18D033204B
:1079D0001AF74ADD09F3F89489EB82DD81E08093A0
:1079E000E00010926F0010928100109285001092BA
:1079F000840085BF15BE5D9A289A0C940000E5E0CE
:107A0000F0E070DDA3E6B2E0C8E063DDCA95E9F717
:107A1000A7DE84EAB0DE80E0AEDEB6DEAADE85EA6E
:107A2000AADEC4E7D1E0DE0184ECA7DE83818D937A
:107A3000A438D1F7A1DE83818D93A6DE1482AFE254
:107A4000B6E08D8117D08C8115D08E8113D09889A6
:107A500092708A8119F08F7184FF80560BD08981D2
:107A600009D0888107D0992321F08A818695807179
:107A700002D053CD00D09E01DD91CD91CD59D94F8B
:107A8000FD91ED91ED59FE4F41915191549F829599
:107A9000682F6F70609DE00DF11DBE01152E8E01E7
:107AA00003561640143050F401900882C058DF4F3E
:107AB0001A94A9F7EB0121964A9579F7E9010895FF
:107AC00048D107C009D102C0AA2039F044D182FFB1
:107AD000FBCF85FFF7CF8091F1000895082E83E05A
:107AE00039D185FD07C02ED102C0AA2049F033D17B
:107AF00080FFFBCF0092F1005D9884E680935001F7
:107B0000089527D182FFEAC0289884E68093510126
:107B1000D7DF182F853431F422248EE7382E8FDCFE
:107B20008DE0C5C0843511F4CBDFFACF8C34C1F3BE
:107B30008035B1F3843711F480E0B9C0813429F481
:107B4000BFDF582EBDDF482EEBCF833539F4E6E991
:107B5000F7E78591C3DFED39E1F7AAC0863521F457
:107B600082E3BCDF81E3A3C08A3649F48FE9C1DC3C
:107B7000C3E0C1DCB3DFCA95E1F7C9DC99C0833744
:107B800031F487E8ABDF85E9A9DF8EE190C082366A
:107B900031F489E5A3DF80E0A1DF80E888C082348A
:107BA00019F0873609F06FC033248ADFD82F88DFB9
:107BB000C82F86DF082F8354843008F077C006343E
:107BC00011F4440C551CF20110926F001736B9F4F1
:107BD000033489F483E087DC8EDC8EB51EBC7EDF47
:107BE0000DB42197D1F793DC08C0063411F48591C8
:107BF00001C02BDC73DF2197C2F72F013CC0033497
:107C0000A9F4E11104C06BDC88ED6DDC7ADC67DC83
:107C100082E069DC55DF0DB48EBDCA95D9F7319687
:107C20006BDC6FDCDA9569F72F0123C00634C1F4F1
:107C30009F01F437A8F4C6D113C042DF063461F4C3
:107C4000C0FB46F0F43728F4182E81E087BFE89592
:107C500011243296082E04C0043409F401C0F9DB63
:107C600021975AF7063429F42F01F901F43708F463
:107C7000A7D18DE033DF063411F45694479482E0A7
:107C800080936F0015C08237E1E049F08634E0E070
:107C900031F08E34E3E019F0813531F4E2E0F0E0C8
:107CA00089E087BF849103C08B3111F08FE316DF29
:107CB00083E0BBDB47D095FF03C009C0AA2071F069
:107CC0004AD080FFFBCF3ED002C0AA2039F043D07B
:107CD00080FFFBCF84E0A9DB8BE735C00895E4E5A6
:107CE000F1E067E090915B0180915C01913231F0AD
:107CF000913A71F5813261F550D173C0823241F110
:107D0000803231F54AD1AA20E9F08530D9F023D06C
:107D100083FD18C082FFF7CF04C0DDDE8193615080
:107D200031F09091F3008091F200892BB1F7D4DF0C
:107D3000611549F704C0AA2029F0853019F00BD04D
:107D400080FFF9CF8EE79091E80089238093E800C7
:107D5000089584E06ADB8091E80008958091E20054
:107D60000895FCDF8E7F80618093E200089582E0B9
:107D700061EC09D083E061E802D084E060E842E190
:107D800003C080E060E042E050DB81E007D0109269
:107D9000ED006093EC004093ED0008959091EB00AE
:107DA000892B8093EB00089560E0923029F09130A8
:107DB00029F4E0E062E102C0E2E16EE3F1E008955F
:107DC00080915B0188234CF402C0AA20C1F3C3DF79
:107DD00082FFFBCF81CFAA2091F3BDDF80FFFBCFD5
:107DE000B1CF40916101509162014617510520F0D9
:107DF000462F611509F4A6DF50E022C0AA2061F1E8
:107E0000853051F1A8DF83FD67CFA5DF82FD21C05A
:107E100080FF16C03091F3002091F20006C08191DE
:107E20008093F10041502F5F3F4F411519F02830EA
:107E30003105A8F350E02830310509F451E082DF24
:107E40004115E1F65523D1F604C0AA2029F085306A
:107E500019F081DF82FFF9CF3FCFEBE5F1E03BDEA8
:107E60008193E336E1F73BDF76DF83FF91C08091BA
:107E70005B0190915C01913009F170F09330F1F069
:107E8000953009F444C0963009F456C0983009F48E
:107E900060C0993059F767C0823841F780915F011F
:107EA000C3DA2091EB001092E90077D02295269555
:107EB00021702093F1001092F10052C0882311F03C
:107EC0008230A1F68F71823089F680915D0188231E
:107ED000D1F420915F01277049F22093E90080914D
:107EE000EB0080FF10C0933011F480E20BC080E102
:107EF00055DF81E0880F2A95E9F78093EA00109218
:107F0000EA0088E04BDF1092E90047D02AC08823BE
:107F100091F410915D0110680FB7F8943ED050DFD6
:107F20001ADF80FFFDCF1093E300103883E009F4DF
:107F300082E0A82E0FBF2CC08058823048F5809177
:107F40005D0190915E0130DF603011F126D049DF94
:107F50001FC08038E9F421D0809153018093F10053
:107F6000F1DE2EDF15C0882399F490915D019230E7
:107F700078F49093530111D023DF8091530188232B
:107F800021F48091E30091E087FD94E0A92EEFDEDB
:107F9000E2DE83FF089580E201DF87EFD4CEA3E61F
:107FA000B1E0F437B8F40ED090E40D901D9081E06C
:107FB00087BFE89532969A95C1F71124E058F040B2
:107FC00085E001C083E001D081E187BFE89507B675
:067FD00000FCFDCF089546
:067FFA003231D2CFFBDCA6
:040000030000740085
:00000001FF
